:020000020000FC
:1000000015C069C00000000000000000ACC0000086
:10001000AEC0B9C000000000000000000D0A626B15
:10002000316E31703431307230350D0A04E00EBF5C
:100030000FE50DBF01E00FBB0FEF0EBBE09A0DB354
:100040000F3F09F001BF04E00EBF0FE50DBF06E44E
:1000500008BB06EF07BB00E005BB00E004BB00E007
:1000600002BB00E001BB02E003BF02E00EBD772748
:10007000882799278AD202E3B02EF9D0F8D0CBD0C6
:10008000EAD0CCD0E8D0CDD0E6D002E3302E0CEED2
:10009000202E00E0C02ED02E05E108BF09BF7894C5
:1000A00003E005BF00E40BBF2AE083FFFECF009111
:1000B000790010917A00877F025E1440A8F72A9594
:1000C000A1F7F894B1D0B0D0AFD078940EE10093FE
:1000D0007B0078D17BC21FB644274BBF45B740FF9A
:1000E0001DC0829B3CC042E045BF4CB55DB5742E3F
:1000F000852E9F7B60917700461B60917800560BA0
:10010000483A61E6560730F4483863E1560710F084
:10011000906425C0BB2019F1BA9421C082991FC0F8
:1001200043E045BF83FD1BC04CB55DB540937700F0
:100130005093780096FF13C09F7B4719580940934E
:10014000790050937A00483968E0560718F7403232
:1001500063E05607F8F2886042E3B42E00C050E432
:100160005BBF1FBE18951FB67E7F1FBE18951FB6BA
:100170007068EE2009F0EA94BB2011F4FF2701C05B
:10018000BA941FBE18951FB676FD26C0906145999A
:100190009F7E422D562D541730F43A9459F452E371
:1001A000352E4A9506C031F03A9421F458E2352EA6
:1001B0004395242E706474FF03C081FFC79807C065
:1001C00075FF03C081FFC49802C081FFC598422D0E
:1001D0004C59409542BF1BC0422D42BF7F7B74FFEC
:1001E00003C080FFC79A07C075FF03C080FFC49A91
:1001F00002C080FFC59A4D3918F482608E7F07C017
:100200004C3E18F08D7F816002C08D7F8E7F93FD04
:1002100081601FBE189538EC10E509C034EB14E678
:1002200006C030EA18E703C034E618EC00C0002727
:1002300002BFC298C49A02B70032E9F7C29AC498C2
:1002400028E0002702BF02B70317E9F72A95C9F78C
:100250001A9569F708951FE028E0002702BF02B74A
:100260000F3FE9F72A95C9F71A95B1F7089510E8F5
:1002700028E0002702BF02B70F3FE9F72A95C9F728
:100280001A95B1F7089530E03BBF30E03EBD32E053
:100290000CB51DB53EBD08958F7E83FF17C000913C
:1002A000790010917A00877F025E144010F40027D5
:1002B00011271695079516950795202F26952695B3
:1002C000021B202F045608F024E6F22F08958F7D9C
:1002D00077FF17C07F7772FF06C07B7F4C2D4330BE
:1002E00088F4C39403C0CC2009F0CA9471FF06C0FF
:1002F0007D7F4D2D443628F4D39403C0DD2009F0D2
:10030000DA940895F89492CE0F2F0D1908F403E1B2
:1003100010916600112321F410916500103438F01B
:100320009160926019E1011798F0012F11C095FFBB
:1003300005C029E1021710F0022F0AC0103238F070
:100340009E7F926012E3011718F0012F01C09C7F7D
:100350000095602E08958F7B20916C0010916B00AA
:1003600000916A00011B00936A0000916B00020B70
:1003700000936B0000916C00004000936C00209192
:100380006900109168000091670026951795079500
:100390002695179507952093690020936800209370
:1003A000670020916A00200F20936A0020916B0063
:1003B000211F20936B0000E020916C00201F2093F0
:1003C0006C000895C0E8DBEBC0937100D09372001D
:1003D0002FEF3FE120936D0030936E0020936F006C
:1003E00030937000E1E0E09366003FEF30936500EA
:1003F0002FEF20936400089546DF00936000109370
:1004000061000C0F1D1F35E039BF1BBD0ABD7160B7
:1004100035E139BF30E43BBF0091640010916500C5
:10042000E09166000093730010937400EE2329F0AE
:100430003FEF3093730030937400E695179507955E
:10044000E695179507952091640030916500E0913D
:100450006600201B310BE0400091600010916100AC
:10046000C0916200D091630000936200109363001A
:100470000C1B1D0B0093750010937600200F311F8D
:1004800010E0E11FEE2361F4332321F0313041F419
:100490002C3430F431E02CE4FF2011F40FEFF02E77
:1004A0002093640030936500E0936600E23008F02A
:1004B00099DF00916700020F0093670000916800C8
:1004C000031F00936800009169000E1F00936900EC
:1004D000E69537952795E69537952795E6953795CF
:1004E0002795E6953795279520936D0030936E00FC
:1004F00020936F00309370000895C0916D00D091EB
:100500006E007ADF089570FDFECF379800B708605F
:1005100000BFD0917400C0917300B5DE0C0F1D1F99
:1005200035E039BF1BBD0ABD716035E139BF30E42C
:100530003BBF0895A8DEC0916F00D09170000C0FF2
:100540001D1F25E029BF1BBD0ABD716025E129BF24
:1005500030E43BBF84FDA0DE85FDB9DE87FDD4DE3F
:1005600086FDF9DE70FDFECF0895C0917100D09137
:10057000720042DF0CB50F70D01BDC3808F4DBEBE7
:10058000D093720014D013D00895F3E10CEE202E16
:10059000602E00E005BB00E002BB02E3302E81606C
:1005A000977F9062089504E00A95F1F7089576FD2B
:1005B000FECF76FFFECF0895089512E301C015E047
:1005C000002702BF02B70117E9F70895DEDFF4DF65
:1005D00063DEF431E8F304E10095602E379800B74C
:1005E000086000BF332700E005BB00E002BBE7DF87
:1005F0003AD13FD19B7F00E000937C0008E2E02EDF
:10060000E1DEB3DF94FF10C070FD02C0946013C040
:10061000CEDF94FDF9CF00E000937C00F6D0FBD054
:100620000BD13ADEA2DF31C070FD02C0946003C07E
:10063000BEDF94FFF9CFE9D098DF94FD08C070FDCC
:1006400002C094600BC0B3DF94FFF9CF07C070FD08
:1006500002C0946003C0ABDF94FDF9CFDCD01CDE98
:1006600084DF94FF08C070FD02C094600BC09FDF60
:1006700094FDF9CF07C070FD02C0946003C097DFFE
:1006800094FFF9CFD9D040DE70DF94FD08C070FD33
:1006900002C094600BC08BDF94FFF9CF07C070FDE0
:1006A00002C0946003C083DF94FDF9CFCBD05DDF3F
:1006B00094FF08C070FD02C094600BC078DF94FD09
:1006C000F9CF07C070FD02C0946003C070DF94FFD3
:1006D000F9CFC9D0FCDD49DF94FD08C070FD02C030
:1006E00094600BC064DF94FFF9CF07C070FD02C0B7
:1006F000946003C05CDF94FDF9CFBBD0022D0C3EAB
:1007000009F464CFEE2009F463CF00916600002362
:1007100021F400916500003250F000917C0092FDC0
:100720000027039500937C009B7F0C3330F00FEF84
:10073000F02EE3DEEADE9F7D02C017DF63CF55D0E7
:1007400070FF41C05AD070FF3EC08064F3DE5DD0C0
:10075000D4DED9DE52D070FF36C047D070FF33C030
:100760008061E8DE58D0C9DECEDE3FD070FF2BC0FE
:1007700044D070FF28C08068DDDE5ED0BEDEC3DE00
:100780003CD070FF20C031D070FF1DC0D3DE5AD0E6
:10079000B4DEB9DE2AD070FF16C02FD070FF13C0B0
:1007A0008062C8DE60D0A9DEAEDE27D070FF0BC04D
:1007B0001CD070FF08C0BEDE5CD09FDEA4DE0091BE
:1007C0006600002319F09062977F02CF977FFF2089
:1007D00041F0FA9429F00F2D013011F0023009F4A4
:1007E0009860ADCFF894D1DE21CC70FF0895459B81
:1007F000FCCFD9DE459BF9CF089570FF0895459948
:10080000FCCFD1DE4599F9CF0895C29A80FFC198F7
:1008100003E007B9089504E109BF00007F7D7F7EF2
:1008200081FD02C076FD03C0C79880FFC59A05E12F
:1008300009BF04E007B90895C19A80FFC69802E095
:1008400007B9089504E109BF000070627F7E81FD51
:1008500002C076FD03C0C59880FFC49A05E109BFB8
:1008600003E007B90895C69A80FFC29804E007B96B
:10087000089504E109BF00007F7D706181FD02C021
:1008800076FD03C0C49880FFC79A05E109BF02E066
:0408900007B9089507
:00000001FF
